Archive member included to satisfy reference by file (symbol)

c:/program files (x86)/atmel/studio/7.0/toolchain/arm/arm-gnu-toolchain/bin/../lib/gcc/arm-none-eabi/6.3.1/thumb/v6-m\libgcc.a(_udivsi3.o)
                              hpl/core/hpl_core_m0plus_base.o (__aeabi_uidiv)
c:/program files (x86)/atmel/studio/7.0/toolchain/arm/arm-gnu-toolchain/bin/../lib/gcc/arm-none-eabi/6.3.1/thumb/v6-m\libgcc.a(_dvmd_tls.o)
                              c:/program files (x86)/atmel/studio/7.0/toolchain/arm/arm-gnu-toolchain/bin/../lib/gcc/arm-none-eabi/6.3.1/thumb/v6-m\libgcc.a(_udivsi3.o) (__aeabi_idiv0)
c:/program files (x86)/atmel/studio/7.0/toolchain/arm/arm-gnu-toolchain/bin/../lib/gcc/arm-none-eabi/6.3.1/thumb/v6-m\libgcc.a(_aeabi_uldivmod.o)
                              hpl/sercom/hpl_sercom.o (__aeabi_uldivmod)
c:/program files (x86)/atmel/studio/7.0/toolchain/arm/arm-gnu-toolchain/bin/../lib/gcc/arm-none-eabi/6.3.1/thumb/v6-m\libgcc.a(_muldi3.o)
                              hpl/sercom/hpl_sercom.o (__aeabi_lmul)
c:/program files (x86)/atmel/studio/7.0/toolchain/arm/arm-gnu-toolchain/bin/../lib/gcc/arm-none-eabi/6.3.1/thumb/v6-m\libgcc.a(_fixunsdfsi.o)
                              hpl/sercom/hpl_sercom.o (__aeabi_d2uiz)
c:/program files (x86)/atmel/studio/7.0/toolchain/arm/arm-gnu-toolchain/bin/../lib/gcc/arm-none-eabi/6.3.1/thumb/v6-m\libgcc.a(_udivmoddi4.o)
                              c:/program files (x86)/atmel/studio/7.0/toolchain/arm/arm-gnu-toolchain/bin/../lib/gcc/arm-none-eabi/6.3.1/thumb/v6-m\libgcc.a(_aeabi_uldivmod.o) (__udivmoddi4)
c:/program files (x86)/atmel/studio/7.0/toolchain/arm/arm-gnu-toolchain/bin/../lib/gcc/arm-none-eabi/6.3.1/thumb/v6-m\libgcc.a(divdf3.o)
                              hpl/sercom/hpl_sercom.o (__aeabi_ddiv)
c:/program files (x86)/atmel/studio/7.0/toolchain/arm/arm-gnu-toolchain/bin/../lib/gcc/arm-none-eabi/6.3.1/thumb/v6-m\libgcc.a(muldf3.o)
                              hpl/sercom/hpl_sercom.o (__aeabi_dmul)
c:/program files (x86)/atmel/studio/7.0/toolchain/arm/arm-gnu-toolchain/bin/../lib/gcc/arm-none-eabi/6.3.1/thumb/v6-m\libgcc.a(subdf3.o)
                              hpl/sercom/hpl_sercom.o (__aeabi_dsub)
c:/program files (x86)/atmel/studio/7.0/toolchain/arm/arm-gnu-toolchain/bin/../lib/gcc/arm-none-eabi/6.3.1/thumb/v6-m\libgcc.a(fixdfsi.o)
                              c:/program files (x86)/atmel/studio/7.0/toolchain/arm/arm-gnu-toolchain/bin/../lib/gcc/arm-none-eabi/6.3.1/thumb/v6-m\libgcc.a(_fixunsdfsi.o) (__aeabi_d2iz)
c:/program files (x86)/atmel/studio/7.0/toolchain/arm/arm-gnu-toolchain/bin/../lib/gcc/arm-none-eabi/6.3.1/thumb/v6-m\libgcc.a(floatsidf.o)
                              hpl/sercom/hpl_sercom.o (__aeabi_i2d)
c:/program files (x86)/atmel/studio/7.0/toolchain/arm/arm-gnu-toolchain/bin/../lib/gcc/arm-none-eabi/6.3.1/thumb/v6-m\libgcc.a(floatunsidf.o)
                              hpl/sercom/hpl_sercom.o (__aeabi_ui2d)
c:/program files (x86)/atmel/studio/7.0/toolchain/arm/arm-gnu-toolchain/bin/../lib/gcc/arm-none-eabi/6.3.1/thumb/v6-m\libgcc.a(_arm_cmpdf2.o)
                              c:/program files (x86)/atmel/studio/7.0/toolchain/arm/arm-gnu-toolchain/bin/../lib/gcc/arm-none-eabi/6.3.1/thumb/v6-m\libgcc.a(_fixunsdfsi.o) (__aeabi_dcmpge)
c:/program files (x86)/atmel/studio/7.0/toolchain/arm/arm-gnu-toolchain/bin/../lib/gcc/arm-none-eabi/6.3.1/thumb/v6-m\libgcc.a(_clzsi2.o)
                              c:/program files (x86)/atmel/studio/7.0/toolchain/arm/arm-gnu-toolchain/bin/../lib/gcc/arm-none-eabi/6.3.1/thumb/v6-m\libgcc.a(divdf3.o) (__clzsi2)
c:/program files (x86)/atmel/studio/7.0/toolchain/arm/arm-gnu-toolchain/bin/../lib/gcc/arm-none-eabi/6.3.1/thumb/v6-m\libgcc.a(_clzdi2.o)
                              c:/program files (x86)/atmel/studio/7.0/toolchain/arm/arm-gnu-toolchain/bin/../lib/gcc/arm-none-eabi/6.3.1/thumb/v6-m\libgcc.a(_udivmoddi4.o) (__clzdi2)
c:/program files (x86)/atmel/studio/7.0/toolchain/arm/arm-gnu-toolchain/bin/../lib/gcc/arm-none-eabi/6.3.1/thumb/v6-m\libgcc.a(eqdf2.o)
                              c:/program files (x86)/atmel/studio/7.0/toolchain/arm/arm-gnu-toolchain/bin/../lib/gcc/arm-none-eabi/6.3.1/thumb/v6-m\libgcc.a(_arm_cmpdf2.o) (__eqdf2)
c:/program files (x86)/atmel/studio/7.0/toolchain/arm/arm-gnu-toolchain/bin/../lib/gcc/arm-none-eabi/6.3.1/thumb/v6-m\libgcc.a(gedf2.o)
                              c:/program files (x86)/atmel/studio/7.0/toolchain/arm/arm-gnu-toolchain/bin/../lib/gcc/arm-none-eabi/6.3.1/thumb/v6-m\libgcc.a(_arm_cmpdf2.o) (__gedf2)
c:/program files (x86)/atmel/studio/7.0/toolchain/arm/arm-gnu-toolchain/bin/../lib/gcc/arm-none-eabi/6.3.1/thumb/v6-m\libgcc.a(ledf2.o)
                              c:/program files (x86)/atmel/studio/7.0/toolchain/arm/arm-gnu-toolchain/bin/../lib/gcc/arm-none-eabi/6.3.1/thumb/v6-m\libgcc.a(_arm_cmpdf2.o) (__ledf2)
c:/program files (x86)/atmel/studio/7.0/toolchain/arm/arm-gnu-toolchain/bin/../lib/gcc/arm-none-eabi/6.3.1/../../../../arm-none-eabi/lib/thumb/v6-m\libc_nano.a(lib_a-exit.o)
                              c:/program files (x86)/atmel/studio/7.0/toolchain/arm/arm-gnu-toolchain/bin/../lib/gcc/arm-none-eabi/6.3.1/../../../../arm-none-eabi/lib/thumb/v6-m/crt0.o (exit)
c:/program files (x86)/atmel/studio/7.0/toolchain/arm/arm-gnu-toolchain/bin/../lib/gcc/arm-none-eabi/6.3.1/../../../../arm-none-eabi/lib/thumb/v6-m\libc_nano.a(lib_a-impure.o)
                              c:/program files (x86)/atmel/studio/7.0/toolchain/arm/arm-gnu-toolchain/bin/../lib/gcc/arm-none-eabi/6.3.1/../../../../arm-none-eabi/lib/thumb/v6-m\libc_nano.a(lib_a-exit.o) (_global_impure_ptr)
c:/program files (x86)/atmel/studio/7.0/toolchain/arm/arm-gnu-toolchain/bin/../lib/gcc/arm-none-eabi/6.3.1/../../../../arm-none-eabi/lib/thumb/v6-m\libc_nano.a(lib_a-init.o)
                              c:/program files (x86)/atmel/studio/7.0/toolchain/arm/arm-gnu-toolchain/bin/../lib/gcc/arm-none-eabi/6.3.1/../../../../arm-none-eabi/lib/thumb/v6-m/crt0.o (__libc_init_array)
c:/program files (x86)/atmel/studio/7.0/toolchain/arm/arm-gnu-toolchain/bin/../lib/gcc/arm-none-eabi/6.3.1/../../../../arm-none-eabi/lib/thumb/v6-m\libc_nano.a(lib_a-memcpy-stub.o)
                              hpl/usb/hpl_usb.o (memcpy)
c:/program files (x86)/atmel/studio/7.0/toolchain/arm/arm-gnu-toolchain/bin/../lib/gcc/arm-none-eabi/6.3.1/../../../../arm-none-eabi/lib/thumb/v6-m\libc_nano.a(lib_a-memset.o)
                              c:/program files (x86)/atmel/studio/7.0/toolchain/arm/arm-gnu-toolchain/bin/../lib/gcc/arm-none-eabi/6.3.1/../../../../arm-none-eabi/lib/thumb/v6-m/crt0.o (memset)
c:/program files (x86)/atmel/studio/7.0/toolchain/arm/arm-gnu-toolchain/bin/../lib/gcc/arm-none-eabi/6.3.1/../../../../arm-none-eabi/lib/thumb/v6-m\libc_nano.a(lib_a-printf.o)
                              hal/utils/src/utils_syscalls.o (printf)
c:/program files (x86)/atmel/studio/7.0/toolchain/arm/arm-gnu-toolchain/bin/../lib/gcc/arm-none-eabi/6.3.1/../../../../arm-none-eabi/lib/thumb/v6-m\libc_nano.a(lib_a-findfp.o)
                              c:/program files (x86)/atmel/studio/7.0/toolchain/arm/arm-gnu-toolchain/bin/../lib/gcc/arm-none-eabi/6.3.1/../../../../arm-none-eabi/lib/thumb/v6-m\libc_nano.a(lib_a-printf.o) (__sinit)
c:/program files (x86)/atmel/studio/7.0/toolchain/arm/arm-gnu-toolchain/bin/../lib/gcc/arm-none-eabi/6.3.1/../../../../arm-none-eabi/lib/thumb/v6-m\libc_nano.a(lib_a-fwalk.o)
                              c:/program files (x86)/atmel/studio/7.0/toolchain/arm/arm-gnu-toolchain/bin/../lib/gcc/arm-none-eabi/6.3.1/../../../../arm-none-eabi/lib/thumb/v6-m\libc_nano.a(lib_a-findfp.o) (_fwalk)
c:/program files (x86)/atmel/studio/7.0/toolchain/arm/arm-gnu-toolchain/bin/../lib/gcc/arm-none-eabi/6.3.1/../../../../arm-none-eabi/lib/thumb/v6-m\libc_nano.a(lib_a-nano-mallocr.o)
                              c:/program files (x86)/atmel/studio/7.0/toolchain/arm/arm-gnu-toolchain/bin/../lib/gcc/arm-none-eabi/6.3.1/../../../../arm-none-eabi/lib/thumb/v6-m\libc_nano.a(lib_a-findfp.o) (_malloc_r)
c:/program files (x86)/atmel/studio/7.0/toolchain/arm/arm-gnu-toolchain/bin/../lib/gcc/arm-none-eabi/6.3.1/../../../../arm-none-eabi/lib/thumb/v6-m\libc_nano.a(lib_a-nano-vfprintf.o)
                              c:/program files (x86)/atmel/studio/7.0/toolchain/arm/arm-gnu-toolchain/bin/../lib/gcc/arm-none-eabi/6.3.1/../../../../arm-none-eabi/lib/thumb/v6-m\libc_nano.a(lib_a-printf.o) (_vfprintf_r)
c:/program files (x86)/atmel/studio/7.0/toolchain/arm/arm-gnu-toolchain/bin/../lib/gcc/arm-none-eabi/6.3.1/../../../../arm-none-eabi/lib/thumb/v6-m\libc_nano.a(lib_a-nano-vfprintf_i.o)
                              c:/program files (x86)/atmel/studio/7.0/toolchain/arm/arm-gnu-toolchain/bin/../lib/gcc/arm-none-eabi/6.3.1/../../../../arm-none-eabi/lib/thumb/v6-m\libc_nano.a(lib_a-nano-vfprintf.o) (_printf_i)
c:/program files (x86)/atmel/studio/7.0/toolchain/arm/arm-gnu-toolchain/bin/../lib/gcc/arm-none-eabi/6.3.1/../../../../arm-none-eabi/lib/thumb/v6-m\libc_nano.a(lib_a-sbrkr.o)
                              c:/program files (x86)/atmel/studio/7.0/toolchain/arm/arm-gnu-toolchain/bin/../lib/gcc/arm-none-eabi/6.3.1/../../../../arm-none-eabi/lib/thumb/v6-m\libc_nano.a(lib_a-nano-mallocr.o) (_sbrk_r)
c:/program files (x86)/atmel/studio/7.0/toolchain/arm/arm-gnu-toolchain/bin/../lib/gcc/arm-none-eabi/6.3.1/../../../../arm-none-eabi/lib/thumb/v6-m\libc_nano.a(lib_a-stdio.o)
                              c:/program files (x86)/atmel/studio/7.0/toolchain/arm/arm-gnu-toolchain/bin/../lib/gcc/arm-none-eabi/6.3.1/../../../../arm-none-eabi/lib/thumb/v6-m\libc_nano.a(lib_a-findfp.o) (__sread)
c:/program files (x86)/atmel/studio/7.0/toolchain/arm/arm-gnu-toolchain/bin/../lib/gcc/arm-none-eabi/6.3.1/../../../../arm-none-eabi/lib/thumb/v6-m\libc_nano.a(lib_a-wbuf.o)
                              c:/program files (x86)/atmel/studio/7.0/toolchain/arm/arm-gnu-toolchain/bin/../lib/gcc/arm-none-eabi/6.3.1/../../../../arm-none-eabi/lib/thumb/v6-m\libc_nano.a(lib_a-nano-vfprintf.o) (__swbuf_r)
c:/program files (x86)/atmel/studio/7.0/toolchain/arm/arm-gnu-toolchain/bin/../lib/gcc/arm-none-eabi/6.3.1/../../../../arm-none-eabi/lib/thumb/v6-m\libc_nano.a(lib_a-writer.o)
                              c:/program files (x86)/atmel/studio/7.0/toolchain/arm/arm-gnu-toolchain/bin/../lib/gcc/arm-none-eabi/6.3.1/../../../../arm-none-eabi/lib/thumb/v6-m\libc_nano.a(lib_a-stdio.o) (_write_r)
c:/program files (x86)/atmel/studio/7.0/toolchain/arm/arm-gnu-toolchain/bin/../lib/gcc/arm-none-eabi/6.3.1/../../../../arm-none-eabi/lib/thumb/v6-m\libc_nano.a(lib_a-wsetup.o)
                              c:/program files (x86)/atmel/studio/7.0/toolchain/arm/arm-gnu-toolchain/bin/../lib/gcc/arm-none-eabi/6.3.1/../../../../arm-none-eabi/lib/thumb/v6-m\libc_nano.a(lib_a-nano-vfprintf.o) (__swsetup_r)
c:/program files (x86)/atmel/studio/7.0/toolchain/arm/arm-gnu-toolchain/bin/../lib/gcc/arm-none-eabi/6.3.1/../../../../arm-none-eabi/lib/thumb/v6-m\libc_nano.a(lib_a-closer.o)
                              c:/program files (x86)/atmel/studio/7.0/toolchain/arm/arm-gnu-toolchain/bin/../lib/gcc/arm-none-eabi/6.3.1/../../../../arm-none-eabi/lib/thumb/v6-m\libc_nano.a(lib_a-stdio.o) (_close_r)
c:/program files (x86)/atmel/studio/7.0/toolchain/arm/arm-gnu-toolchain/bin/../lib/gcc/arm-none-eabi/6.3.1/../../../../arm-none-eabi/lib/thumb/v6-m\libc_nano.a(lib_a-fflush.o)
                              c:/program files (x86)/atmel/studio/7.0/toolchain/arm/arm-gnu-toolchain/bin/../lib/gcc/arm-none-eabi/6.3.1/../../../../arm-none-eabi/lib/thumb/v6-m\libc_nano.a(lib_a-findfp.o) (_fflush_r)
c:/program files (x86)/atmel/studio/7.0/toolchain/arm/arm-gnu-toolchain/bin/../lib/gcc/arm-none-eabi/6.3.1/../../../../arm-none-eabi/lib/thumb/v6-m\libc_nano.a(lib_a-fvwrite.o)
                              c:/program files (x86)/atmel/studio/7.0/toolchain/arm/arm-gnu-toolchain/bin/../lib/gcc/arm-none-eabi/6.3.1/../../../../arm-none-eabi/lib/thumb/v6-m\libc_nano.a(lib_a-nano-vfprintf.o) (__sfvwrite_r)
c:/program files (x86)/atmel/studio/7.0/toolchain/arm/arm-gnu-toolchain/bin/../lib/gcc/arm-none-eabi/6.3.1/../../../../arm-none-eabi/lib/thumb/v6-m\libc_nano.a(lib_a-lseekr.o)
                              c:/program files (x86)/atmel/studio/7.0/toolchain/arm/arm-gnu-toolchain/bin/../lib/gcc/arm-none-eabi/6.3.1/../../../../arm-none-eabi/lib/thumb/v6-m\libc_nano.a(lib_a-stdio.o) (_lseek_r)
c:/program files (x86)/atmel/studio/7.0/toolchain/arm/arm-gnu-toolchain/bin/../lib/gcc/arm-none-eabi/6.3.1/../../../../arm-none-eabi/lib/thumb/v6-m\libc_nano.a(lib_a-makebuf.o)
                              c:/program files (x86)/atmel/studio/7.0/toolchain/arm/arm-gnu-toolchain/bin/../lib/gcc/arm-none-eabi/6.3.1/../../../../arm-none-eabi/lib/thumb/v6-m\libc_nano.a(lib_a-wsetup.o) (__smakebuf_r)
c:/program files (x86)/atmel/studio/7.0/toolchain/arm/arm-gnu-toolchain/bin/../lib/gcc/arm-none-eabi/6.3.1/../../../../arm-none-eabi/lib/thumb/v6-m\libc_nano.a(lib_a-memchr-stub.o)
                              c:/program files (x86)/atmel/studio/7.0/toolchain/arm/arm-gnu-toolchain/bin/../lib/gcc/arm-none-eabi/6.3.1/../../../../arm-none-eabi/lib/thumb/v6-m\libc_nano.a(lib_a-nano-vfprintf.o) (memchr)
c:/program files (x86)/atmel/studio/7.0/toolchain/arm/arm-gnu-toolchain/bin/../lib/gcc/arm-none-eabi/6.3.1/../../../../arm-none-eabi/lib/thumb/v6-m\libc_nano.a(lib_a-memmove.o)
                              c:/program files (x86)/atmel/studio/7.0/toolchain/arm/arm-gnu-toolchain/bin/../lib/gcc/arm-none-eabi/6.3.1/../../../../arm-none-eabi/lib/thumb/v6-m\libc_nano.a(lib_a-fvwrite.o) (memmove)
c:/program files (x86)/atmel/studio/7.0/toolchain/arm/arm-gnu-toolchain/bin/../lib/gcc/arm-none-eabi/6.3.1/../../../../arm-none-eabi/lib/thumb/v6-m\libc_nano.a(lib_a-mlock.o)
                              c:/program files (x86)/atmel/studio/7.0/toolchain/arm/arm-gnu-toolchain/bin/../lib/gcc/arm-none-eabi/6.3.1/../../../../arm-none-eabi/lib/thumb/v6-m\libc_nano.a(lib_a-nano-mallocr.o) (__malloc_lock)
c:/program files (x86)/atmel/studio/7.0/toolchain/arm/arm-gnu-toolchain/bin/../lib/gcc/arm-none-eabi/6.3.1/../../../../arm-none-eabi/lib/thumb/v6-m\libc_nano.a(lib_a-nano-freer.o)
                              c:/program files (x86)/atmel/studio/7.0/toolchain/arm/arm-gnu-toolchain/bin/../lib/gcc/arm-none-eabi/6.3.1/../../../../arm-none-eabi/lib/thumb/v6-m\libc_nano.a(lib_a-wsetup.o) (_free_r)
c:/program files (x86)/atmel/studio/7.0/toolchain/arm/arm-gnu-toolchain/bin/../lib/gcc/arm-none-eabi/6.3.1/../../../../arm-none-eabi/lib/thumb/v6-m\libc_nano.a(lib_a-nano-reallocr.o)
                              c:/program files (x86)/atmel/studio/7.0/toolchain/arm/arm-gnu-toolchain/bin/../lib/gcc/arm-none-eabi/6.3.1/../../../../arm-none-eabi/lib/thumb/v6-m\libc_nano.a(lib_a-fvwrite.o) (_realloc_r)
c:/program files (x86)/atmel/studio/7.0/toolchain/arm/arm-gnu-toolchain/bin/../lib/gcc/arm-none-eabi/6.3.1/../../../../arm-none-eabi/lib/thumb/v6-m\libc_nano.a(lib_a-readr.o)
                              c:/program files (x86)/atmel/studio/7.0/toolchain/arm/arm-gnu-toolchain/bin/../lib/gcc/arm-none-eabi/6.3.1/../../../../arm-none-eabi/lib/thumb/v6-m\libc_nano.a(lib_a-stdio.o) (_read_r)
c:/program files (x86)/atmel/studio/7.0/toolchain/arm/arm-gnu-toolchain/bin/../lib/gcc/arm-none-eabi/6.3.1/../../../../arm-none-eabi/lib/thumb/v6-m\libc_nano.a(lib_a-reent.o)
                              c:/program files (x86)/atmel/studio/7.0/toolchain/arm/arm-gnu-toolchain/bin/../lib/gcc/arm-none-eabi/6.3.1/../../../../arm-none-eabi/lib/thumb/v6-m\libc_nano.a(lib_a-sbrkr.o) (errno)
c:/program files (x86)/atmel/studio/7.0/toolchain/arm/arm-gnu-toolchain/bin/../lib/gcc/arm-none-eabi/6.3.1/../../../../arm-none-eabi/lib/thumb/v6-m\libc_nano.a(lib_a-fstatr.o)
                              c:/program files (x86)/atmel/studio/7.0/toolchain/arm/arm-gnu-toolchain/bin/../lib/gcc/arm-none-eabi/6.3.1/../../../../arm-none-eabi/lib/thumb/v6-m\libc_nano.a(lib_a-makebuf.o) (_fstat_r)
c:/program files (x86)/atmel/studio/7.0/toolchain/arm/arm-gnu-toolchain/bin/../lib/gcc/arm-none-eabi/6.3.1/../../../../arm-none-eabi/lib/thumb/v6-m\libc_nano.a(lib_a-isattyr.o)
                              c:/program files (x86)/atmel/studio/7.0/toolchain/arm/arm-gnu-toolchain/bin/../lib/gcc/arm-none-eabi/6.3.1/../../../../arm-none-eabi/lib/thumb/v6-m\libc_nano.a(lib_a-makebuf.o) (_isatty_r)
c:/program files (x86)/atmel/studio/7.0/toolchain/arm/arm-gnu-toolchain/bin/../lib/gcc/arm-none-eabi/6.3.1/../../../../arm-none-eabi/lib/thumb/v6-m\libc_nano.a(lib_a-nano-msizer.o)
                              c:/program files (x86)/atmel/studio/7.0/toolchain/arm/arm-gnu-toolchain/bin/../lib/gcc/arm-none-eabi/6.3.1/../../../../arm-none-eabi/lib/thumb/v6-m\libc_nano.a(lib_a-nano-reallocr.o) (_malloc_usable_size_r)
c:/program files (x86)/atmel/studio/7.0/toolchain/arm/arm-gnu-toolchain/bin/../lib/gcc/arm-none-eabi/6.3.1/thumb/v6-m\libgcc.a(_divsi3.o)
                              c:/program files (x86)/atmel/studio/7.0/toolchain/arm/arm-gnu-toolchain/bin/../lib/gcc/arm-none-eabi/6.3.1/../../../../arm-none-eabi/lib/thumb/v6-m\libc_nano.a(lib_a-fvwrite.o) (__aeabi_idiv)

Allocating common symbols
Common symbol       size              file

errno               0x4               c:/program files (x86)/atmel/studio/7.0/toolchain/arm/arm-gnu-toolchain/bin/../lib/gcc/arm-none-eabi/6.3.1/../../../../arm-none-eabi/lib/thumb/v6-m\libc_nano.a(lib_a-reent.o)
_irq_table          0x74              hpl/core/hpl_core_m0plus_base.o
SPI_0               0x18              driver_init.o
TIMER_0             0x1c              driver_init.o

Discarded input sections

 .text          0x00000000        0x0 c:/program files (x86)/atmel/studio/7.0/toolchain/arm/arm-gnu-toolchain/bin/../lib/gcc/arm-none-eabi/6.3.1/thumb/v6-m/crti.o
 .data          0x00000000        0x0 c:/program files (x86)/atmel/studio/7.0/toolchain/arm/arm-gnu-toolchain/bin/../lib/gcc/arm-none-eabi/6.3.1/thumb/v6-m/crti.o
 .bss           0x00000000        0x0 c:/program files (x86)/atmel/studio/7.0/toolchain/arm/arm-gnu-toolchain/bin/../lib/gcc/arm-none-eabi/6.3.1/thumb/v6-m/crti.o
 .data          0x00000000        0x4 c:/program files (x86)/atmel/studio/7.0/toolchain/arm/arm-gnu-toolchain/bin/../lib/gcc/arm-none-eabi/6.3.1/thumb/v6-m/crtbegin.o
 .text          0x00000000       0x78 c:/program files (x86)/atmel/studio/7.0/toolchain/arm/arm-gnu-toolchain/bin/../lib/gcc/arm-none-eabi/6.3.1/../../../../arm-none-eabi/lib/thumb/v6-m/crt0.o
 .data          0x00000000        0x0 c:/program files (x86)/atmel/studio/7.0/toolchain/arm/arm-gnu-toolchain/bin/../lib/gcc/arm-none-eabi/6.3.1/../../../../arm-none-eabi/lib/thumb/v6-m/crt0.o
 .bss           0x00000000        0x0 c:/program files (x86)/atmel/studio/7.0/toolchain/arm/arm-gnu-toolchain/bin/../lib/gcc/arm-none-eabi/6.3.1/../../../../arm-none-eabi/lib/thumb/v6-m/crt0.o
 .ARM.extab     0x00000000        0x0 c:/program files (x86)/atmel/studio/7.0/toolchain/arm/arm-gnu-toolchain/bin/../lib/gcc/arm-none-eabi/6.3.1/../../../../arm-none-eabi/lib/thumb/v6-m/crt0.o
 .ARM.exidx     0x00000000        0x8 c:/program files (x86)/atmel/studio/7.0/toolchain/arm/arm-gnu-toolchain/bin/../lib/gcc/arm-none-eabi/6.3.1/../../../../arm-none-eabi/lib/thumb/v6-m/crt0.o
 .ARM.attributes
                0x00000000       0x1b c:/program files (x86)/atmel/studio/7.0/toolchain/arm/arm-gnu-toolchain/bin/../lib/gcc/arm-none-eabi/6.3.1/../../../../arm-none-eabi/lib/thumb/v6-m/crt0.o
 .group         0x00000000        0x8 atmel_start.o
 .group         0x00000000        0x8 atmel_start.o
 .group         0x00000000        0x8 atmel_start.o
 .group         0x00000000        0x8 atmel_start.o
 .group         0x00000000        0x8 atmel_start.o
 .group         0x00000000        0x8 atmel_start.o
 .group         0x00000000        0x8 atmel_start.o
Memory Configuration

Name             Origin             Length             Attributes
rom              0x00000000         0x00008000         xr
ram              0x20000000         0x00001000         xrw
*default*        0x00000000         0xffffffff

Linker script and memory map

LOAD c:/program files (x86)/atmel/studio/7.0/toolchain/arm/arm-gnu-toolchain/bin/../lib/gcc/arm-none-eabi/6.3.1/thumb/v6-m/crti.o
LOAD c:/program files (x86)/atmel/studio/7.0/toolchain/arm/arm-gnu-toolchain/bin/../lib/gcc/arm-none-eabi/6.3.1/thumb/v6-m/crtbegin.o
LOAD c:/program files (x86)/atmel/studio/7.0/toolchain/arm/arm-gnu-toolchain/bin/../lib/gcc/arm-none-eabi/6.3.1/../../../../arm-none-eabi/lib/thumb/v6-m/crt0.o
LOAD atmel_start.o
LOAD Device_Startup/startup_samd21.o
LOAD Device_Startup/system_samd21.o
LOAD driver_init.o
LOAD examples/driver_examples.o
LOAD hal/src/hal_atomic.o
LOAD hal/src/hal_delay.o
LOAD hal/src/hal_gpio.o
LOAD hal/src/hal_init.o
LOAD hal/src/hal_io.o
LOAD hal/src/hal_sleep.o
LOAD hal/src/hal_spi_m_sync.o
LOAD hal/src/hal_timer.o
LOAD hal/src/hal_usb_device.o
LOAD hal/utils/src/utils_assert.o
LOAD hal/utils/src/utils_event.o
LOAD hal/utils/src/utils_list.o
LOAD hal/utils/src/utils_syscalls.o
LOAD hpl/core/hpl_core_m0plus_base.o
LOAD hpl/core/hpl_init.o
LOAD hpl/dmac/hpl_dmac.o
LOAD hpl/gclk/hpl_gclk.o
LOAD hpl/pm/hpl_pm.o
LOAD hpl/rtc/hpl_rtc.o
LOAD hpl/sercom/hpl_sercom.o
LOAD hpl/sysctrl/hpl_sysctrl.o
LOAD hpl/usb/hpl_usb.o
LOAD main.o
START GROUP
LOAD c:/program files (x86)/atmel/studio/7.0/toolchain/arm/arm-gnu-toolchain/bin/../lib/gcc/arm-none-eabi/6.3.1/../../../../arm-none-eabi/lib/thumb/v6-m\libm.a
END GROUP
START GROUP
LOAD c:/program files (x86)/atmel/studio/7.0/toolchain/arm/arm-gnu-toolchain/bin/../lib/gcc/arm-none-eabi/6.3.1/thumb/v6-m\libgcc.a
LOAD c:/program files (x86)/atmel/studio/7.0/toolchain/arm/arm-gnu-toolchain/bin/../lib/gcc/arm-none-eabi/6.3.1/../../../../arm-none-eabi/lib/thumb/v6-m\libc_nano.a
END GROUP
START GROUP
LOAD c:/program files (x86)/atmel/studio/7.0/toolchain/arm/arm-gnu-toolchain/bin/../lib/gcc/arm-none-eabi/6.3.1/thumb/v6-m\libgcc.a
LOAD c:/program files (x86)/atmel/studio/7.0/toolchain/arm/arm-gnu-toolchain/bin/../lib/gcc/arm-none-eabi/6.3.1/../../../../arm-none-eabi/lib/thumb/v6-m\libc_nano.a
END GROUP
LOAD c:/program files (x86)/atmel/studio/7.0/toolchain/arm/arm-gnu-toolchain/bin/../lib/gcc/arm-none-eabi/6.3.1/thumb/v6-m/crtend.o
LOAD c:/program files (x86)/atmel/studio/7.0/toolchain/arm/arm-gnu-toolchain/bin/../lib/gcc/arm-none-eabi/6.3.1/thumb/v6-m/crtn.o
                0x00000400                STACK_SIZE = DEFINED (STACK_SIZE)?STACK_SIZE:DEFINED (__stack_size__)?__stack_size__:0x400

.text           0x00000000     0x1f78
                0x00000000                . = ALIGN (0x4)
                0x00000000                _sfixed = .
 *(.vectors .vectors.*)
 .vectors       0x00000000       0xb4 Device_Startup/startup_samd21.o
                0x00000000                exception_table
 *(.text .text.* .gnu.linkonce.t.*)
 .text          0x000000b4       0x60 c:/program files (x86)/atmel/studio/7.0/toolchain/arm/arm-gnu-toolchain/bin/../lib/gcc/arm-none-eabi/6.3.1/thumb/v6-m/crtbegin.o
 .text.atmel_start_init
                0x00000114        0xc atmel_start.o
                0x00000114                atmel_start_init
 .text.Dummy_Handler
                0x00000120        0x2 Device_Startup/startup_samd21.o
                0x00000120                SVCall_Handler
                0x00000120                DMAC_Handler
                0x00000120                HardFault_Handler
                0x00000120                AC_Handler
                0x00000120                SysTick_Handler
                0x00000120                PendSV_Handler
                0x00000120                SERCOM1_Handler
                0x00000120                ADC_Handler
                0x00000120                NonMaskableInt_Handler
                0x00000120                TCC1_Handler
                0x00000120                SERCOM2_Handler
                0x00000120                TCC0_Handler
                0x00000120                EIC_Handler
                0x00000120                WDT_Handler
                0x00000120                TC4_Handler
                0x00000120                TC3_Handler
                0x00000120                Dummy_Handler
                0x00000120                PM_Handler
                0x00000120                TCC2_Handler
                0x00000120                EVSYS_Handler
                0x00000120                SERCOM3_Handler
                0x00000120                I2S_Handler
                0x00000120                NVMCTRL_Handler
                0x00000120                SERCOM0_Handler
                0x00000120                DAC_Handler
                0x00000120                PTC_Handler
                0x00000120                TC5_Handler
                0x00000120                SYSCTRL_Handler
 *fill*         0x00000122        0x2 
 .text.Reset_Handler
                0x00000124       0xc4 Device_Startup/startup_samd21.o
                0x00000124                Reset_Handler
 .text.TIMER_0_init
                0x000001e8       0x40 driver_init.o
 .text.SPI_0_PORT_init
                0x00000228       0xbc driver_init.o
                0x00000228                SPI_0_PORT_init
 .text.SPI_0_CLOCK_init
                0x000002e4       0x20 driver_init.o
                0x000002e4                SPI_0_CLOCK_init
 .text.SPI_0_init
                0x00000304       0x28 driver_init.o
                0x00000304                SPI_0_init
 .text.USB_0_PORT_init
                0x0000032c       0x90 driver_init.o
                0x0000032c                USB_0_PORT_init
 .text.USB_0_CLOCK_init
                0x000003bc       0x28 driver_init.o
                0x000003bc                USB_0_CLOCK_init
 .text.USB_0_init
                0x000003e4       0x1c driver_init.o
                0x000003e4                USB_0_init
 .text.system_init
                0x00000400      0x18c driver_init.o
                0x00000400                system_init
 .text.atomic_enter_critical
                0x0000058c        0xe hal/src/hal_atomic.o
                0x0000058c                atomic_enter_critical
 .text.atomic_leave_critical
                0x0000059a        0xc hal/src/hal_atomic.o
                0x0000059a                atomic_leave_critical
 *fill*         0x000005a6        0x2 
 .text.spi_m_sync_init
                0x000005a8       0x58 hal/src/hal_spi_m_sync.o
                0x000005a8                spi_m_sync_init
 .text.spi_m_sync_transfer
                0x00000600       0x48 hal/src/hal_spi_m_sync.o
                0x00000600                spi_m_sync_transfer
 .text._spi_m_sync_io_write
                0x00000648       0x3c hal/src/hal_spi_m_sync.o
 .text._spi_m_sync_io_read
                0x00000684       0x3c hal/src/hal_spi_m_sync.o
 .text.timer_add_timer_task
                0x000006c0       0x58 hal/src/hal_timer.o
 .text.timer_process_counted
                0x00000718       0x64 hal/src/hal_timer.o
 .text.timer_init
                0x0000077c       0x44 hal/src/hal_timer.o
                0x0000077c                timer_init
 .text._usb_d_find_ep
                0x000007c0       0x3c hal/src/hal_usb_device.o
 .text.usb_d_dummy_cb_false
                0x000007fc        0x4 hal/src/hal_usb_device.o
 .text.usb_d_cb_trans_more
                0x00000800       0x30 hal/src/hal_usb_device.o
 .text._usb_d_cb_trans_done
                0x00000830      0x144 hal/src/hal_usb_device.o
 .text.usb_d_cb_trans_setup
                0x00000974       0x98 hal/src/hal_usb_device.o
 .text.usb_d_init
                0x00000a0c       0x6c hal/src/hal_usb_device.o
                0x00000a0c                usb_d_init
 .text.assert   0x00000a78        0x8 hal/utils/src/utils_assert.o
                0x00000a78                assert
 .text.is_list_element
                0x00000a80       0x16 hal/utils/src/utils_list.o
                0x00000a80                is_list_element
 *fill*         0x00000a96        0x2 
 .text.list_insert_as_head
                0x00000a98       0x2c hal/utils/src/utils_list.o
                0x00000a98                list_insert_as_head
 .text.list_insert_after
                0x00000ac4        0x8 hal/utils/src/utils_list.o
                0x00000ac4                list_insert_after
 .text.list_remove_head
                0x00000acc       0x12 hal/utils/src/utils_list.o
                0x00000acc                list_remove_head
 *fill*         0x00000ade        0x2 
 .text._init_chip
                0x00000ae0       0x34 hpl/core/hpl_init.o
                0x00000ae0                _init_chip
 .text._gclk_init_generators_by_fref
                0x00000b14       0x5c hpl/gclk/hpl_gclk.o
                0x00000b14                _gclk_init_generators_by_fref
 .text._pm_init
                0x00000b70       0x20 hpl/pm/hpl_pm.o
                0x00000b70                _pm_init
 .text._rtc_timer_interrupt_handler
                0x00000b90       0x1c hpl/rtc/hpl_rtc.o
 .text._timer_init
                0x00000bac       0x5c hpl/rtc/hpl_rtc.o
                0x00000bac                _timer_init
 .text._rtc_get_timer
                0x00000c08        0x4 hpl/rtc/hpl_rtc.o
                0x00000c08                _rtc_get_timer
 .text.RTC_Handler
                0x00000c0c       0x14 hpl/rtc/hpl_rtc.o
                0x00000c0c                RTC_Handler
 .text._sercom_get_hardware_index
                0x00000c20       0x10 hpl/sercom/hpl_sercom.o
 .text._spi_m_sync_init
                0x00000c30      0x1fc hpl/sercom/hpl_sercom.o
                0x00000c30                _spi_m_sync_init
 .text._spi_m_sync_trans
                0x00000e2c      0x114 hpl/sercom/hpl_sercom.o
                0x00000e2c                _spi_m_sync_trans
 .text._sysctrl_init_sources
                0x00000f40       0x4c hpl/sysctrl/hpl_sysctrl.o
                0x00000f40                _sysctrl_init_sources
 .text._sysctrl_init_referenced_generators
                0x00000f8c       0x88 hpl/sysctrl/hpl_sysctrl.o
                0x00000f8c                _sysctrl_init_referenced_generators
 .text._dummy_func_no_return
                0x00001014        0x4 hpl/usb/hpl_usb.o
 .text._usb_load_calib
                0x00001018       0x54 hpl/usb/hpl_usb.o
 .text._usb_d_dev_handle_setup
                0x0000106c       0x8c hpl/usb/hpl_usb.o
 .text._usb_d_dev_handle_stall
                0x000010f8       0x30 hpl/usb/hpl_usb.o
 .text._usb_d_dev_trans_done
                0x00001128       0x28 hpl/usb/hpl_usb.o
 .text._usb_d_dev_trans_stop
                0x00001150       0x7c hpl/usb/hpl_usb.o
 .text._usb_d_dev_handle_trfail
                0x000011cc      0x110 hpl/usb/hpl_usb.o
 .text._usb_d_dev_reset_epts
                0x000012dc       0x54 hpl/usb/hpl_usb.o
 .text._usb_d_dev_in_next
                0x00001330      0x18c hpl/usb/hpl_usb.o
 .text._usb_d_dev_out_next
                0x000014bc      0x204 hpl/usb/hpl_usb.o
 .text._usb_d_dev_handler
                0x000016c0      0x254 hpl/usb/hpl_usb.o
 .text._usb_d_dev_init
                0x00001914       0xa4 hpl/usb/hpl_usb.o
                0x00001914                _usb_d_dev_init
 .text._usb_d_dev_ep_stall
                0x000019b8      0x158 hpl/usb/hpl_usb.o
                0x000019b8                _usb_d_dev_ep_stall
 .text._usb_d_dev_ep_read_req
                0x00001b10       0x78 hpl/usb/hpl_usb.o
                0x00001b10                _usb_d_dev_ep_read_req
 .text._usb_d_dev_ep_trans
                0x00001b88      0x1d8 hpl/usb/hpl_usb.o
                0x00001b88                _usb_d_dev_ep_trans
 .text._usb_d_dev_register_ep_callback
                0x00001d60       0x30 hpl/usb/hpl_usb.o
                0x00001d60                _usb_d_dev_register_ep_callback
 .text.USB_Handler
                0x00001d90        0xc hpl/usb/hpl_usb.o
                0x00001d90                USB_Handler
 .text.main     0x00001d9c       0x38 main.o
                0x00001d9c                main
 .text.__libc_init_array
                0x00001dd4       0x48 c:/program files (x86)/atmel/studio/7.0/toolchain/arm/arm-gnu-toolchain/bin/../lib/gcc/arm-none-eabi/6.3.1/../../../../arm-none-eabi/lib/thumb/v6-m\libc_nano.a(lib_a-init.o)
                0x00001dd4                __libc_init_array
 .text.memcpy   0x00001e1c       0x12 c:/program files (x86)/atmel/studio/7.0/toolchain/arm/arm-gnu-toolchain/bin/../lib/gcc/arm-none-eabi/6.3.1/../../../../arm-none-eabi/lib/thumb/v6-m\libc_nano.a(lib_a-memcpy-stub.o)
                0x00001e1c                memcpy
 .text.memset   0x00001e2e       0x10 c:/program files (x86)/atmel/studio/7.0/toolchain/arm/arm-gnu-toolchain/bin/../lib/gcc/arm-none-eabi/6.3.1/../../../../arm-none-eabi/lib/thumb/v6-m\libc_nano.a(lib_a-memset.o)
                0x00001e2e                memset
 *(.glue_7t)
 .glue_7t       0x00001e3e        0x0 linker stubs
 *(.glue_7)
 .glue_7        0x00001e3e        0x0 linker stubs
 *(.rodata .rodata* .gnu.linkonce.r.*)
 *fill*         0x00001e3e        0x2 
 .rodata.str1.4
                0x00001e40       0x1c hal/src/hal_spi_m_sync.o
 .rodata.str1.4
                0x00001e5c       0x17 hal/src/hal_timer.o
 *fill*         0x00001e73        0x1 
 .rodata.str1.4
                0x00001e74       0x1e hal/utils/src/utils_list.o
 *fill*         0x00001e92        0x2 
 .rodata.str1.4
                0x00001e94       0x15 hpl/rtc/hpl_rtc.o
 *fill*         0x00001ea9        0x3 
 .rodata        0x00001eac       0x4d hpl/sercom/hpl_sercom.o
 *fill*         0x00001ef9        0x3 
 .rodata.str1.4
                0x00001efc       0x1c hpl/sercom/hpl_sercom.o
                                 0x1b (size before relaxing)
 .rodata        0x00001f18       0x2c hpl/usb/hpl_usb.o
 .rodata        0x00001f44       0x13 main.o
                0x00001f44                RGB_pins
                0x00001f4c                B_pins
                0x00001f50                G_pins
                0x00001f54                R_pins
 *(.ARM.extab* .gnu.linkonce.armextab.*)
                0x00001f58                . = ALIGN (0x4)
 *fill*         0x00001f57        0x1 
 *(.init)
 .init          0x00001f58        0x4 c:/program files (x86)/atmel/studio/7.0/toolchain/arm/arm-gnu-toolchain/bin/../lib/gcc/arm-none-eabi/6.3.1/thumb/v6-m/crti.o
                0x00001f58                _init
 .init          0x00001f5c        0x8 c:/program files (x86)/atmel/studio/7.0/toolchain/arm/arm-gnu-toolchain/bin/../lib/gcc/arm-none-eabi/6.3.1/thumb/v6-m/crtn.o
                0x00001f64                . = ALIGN (0x4)
                0x00001f64                __preinit_array_start = .
 *(.preinit_array)
                0x00001f64                __preinit_array_end = .
                0x00001f64                . = ALIGN (0x4)
                0x00001f64                __init_array_start = .
 *(SORT(.init_array.*))
 *(.init_array)
 .init_array    0x00001f64        0x4 c:/program files (x86)/atmel/studio/7.0/toolchain/arm/arm-gnu-toolchain/bin/../lib/gcc/arm-none-eabi/6.3.1/thumb/v6-m/crtbegin.o
                0x00001f68                __init_array_end = .
                0x00001f68                . = ALIGN (0x4)
 *crtbegin.o(.ctors)
 *(EXCLUDE_FILE(*crtend.o) .ctors)
 *(SORT(.ctors.*))
 *crtend.o(.ctors)
                0x00001f68                . = ALIGN (0x4)
 *(.fini)
 .fini          0x00001f68        0x4 c:/program files (x86)/atmel/studio/7.0/toolchain/arm/arm-gnu-toolchain/bin/../lib/gcc/arm-none-eabi/6.3.1/thumb/v6-m/crti.o
                0x00001f68                _fini
 .fini          0x00001f6c        0x8 c:/program files (x86)/atmel/studio/7.0/toolchain/arm/arm-gnu-toolchain/bin/../lib/gcc/arm-none-eabi/6.3.1/thumb/v6-m/crtn.o
                0x00001f74                . = ALIGN (0x4)
                0x00001f74                __fini_array_start = .
 *(.fini_array)
 .fini_array    0x00001f74        0x4 c:/program files (x86)/atmel/studio/7.0/toolchain/arm/arm-gnu-toolchain/bin/../lib/gcc/arm-none-eabi/6.3.1/thumb/v6-m/crtbegin.o
 *(SORT(.fini_array.*))
                0x00001f78                __fini_array_end = .
 *crtbegin.o(.dtors)
 *(EXCLUDE_FILE(*crtend.o) .dtors)
 *(SORT(.dtors.*))
 *crtend.o(.dtors)
                0x00001f78                . = ALIGN (0x4)
                0x00001f78                _efixed = .
                [!provide]                PROVIDE (__exidx_start, .)

.vfp11_veneer   0x00001f78        0x0
 .vfp11_veneer  0x00001f78        0x0 linker stubs

.v4_bx          0x00001f78        0x0
 .v4_bx         0x00001f78        0x0 linker stubs

.iplt           0x00001f78        0x0
 .iplt          0x00001f78        0x0 c:/program files (x86)/atmel/studio/7.0/toolchain/arm/arm-gnu-toolchain/bin/../lib/gcc/arm-none-eabi/6.3.1/thumb/v6-m/crtbegin.o

.eh_frame       0x00001f78        0x0
 .eh_frame      0x00001f78        0x0 c:/program files (x86)/atmel/studio/7.0/toolchain/arm/arm-gnu-toolchain/bin/../lib/gcc/arm-none-eabi/6.3.1/thumb/v6-m/crtbegin.o

.rel.dyn        0x00001f78        0x0
 .rel.iplt      0x00001f78        0x0 c:/program files (x86)/atmel/studio/7.0/toolchain/arm/arm-gnu-toolchain/bin/../lib/gcc/arm-none-eabi/6.3.1/thumb/v6-m/crtbegin.o

.jcr            0x00001f78        0x0
 .jcr           0x00001f78        0x0 c:/program files (x86)/atmel/studio/7.0/toolchain/arm/arm-gnu-toolchain/bin/../lib/gcc/arm-none-eabi/6.3.1/thumb/v6-m/crtbegin.o

.igot.plt       0x00001f78        0x0
 .igot.plt      0x00001f78        0x0 c:/program files (x86)/atmel/studio/7.0/toolchain/arm/arm-gnu-toolchain/bin/../lib/gcc/arm-none-eabi/6.3.1/thumb/v6-m/crtbegin.o

.ARM.exidx
 *(.ARM.exidx* .gnu.linkonce.armexidx.*)
                [!provide]                PROVIDE (__exidx_end, .)
                0x00001f78                . = ALIGN (0x4)
                0x00001f78                _etext = .

.relocate       0x20000000        0x0 load address 0x00001f78
                0x20000000                . = ALIGN (0x4)
                0x20000000                _srelocate = .
 *(.ramfunc .ramfunc.*)
 *(.data .data.*)
                0x20000000                . = ALIGN (0x4)
                0x20000000                _erelocate = .

.bss            0x20000000      0x2bc
                0x20000000                . = ALIGN (0x4)
                0x20000000                _sbss = .
                0x20000000                _szero = .
 *(.bss .bss.*)
 .bss           0x20000000       0x1c c:/program files (x86)/atmel/studio/7.0/toolchain/arm/arm-gnu-toolchain/bin/../lib/gcc/arm-none-eabi/6.3.1/thumb/v6-m/crtbegin.o
 .bss           0x2000001c       0x80 hal/src/hal_usb_device.o
 .bss           0x2000009c        0x4 hpl/rtc/hpl_rtc.o
 .bss           0x200000a0      0x1e8 hpl/usb/hpl_usb.o
 *(COMMON)
 COMMON         0x20000288       0x34 driver_init.o
                0x20000288                SPI_0
                0x200002a0                TIMER_0
                0x200002bc                . = ALIGN (0x4)
                0x200002bc                _ebss = .
                0x200002bc                _ezero = .

.stack          0x200002bc      0x404
                0x200002c0                . = ALIGN (0x8)
 *fill*         0x200002bc        0x4 
                0x200002c0                _sstack = .
                0x200006c0                . = (. + STACK_SIZE)
 *fill*         0x200002c0      0x400 
                0x200006c0                . = ALIGN (0x8)
                0x200006c0                _estack = .
                0x200006c0                . = ALIGN (0x4)
                0x200006c0                _end = .
OUTPUT(ConwayVGA.elf elf32-littlearm)

.ARM.attributes
                0x00000000       0x28
 .ARM.attributes
                0x00000000       0x1e c:/program files (x86)/atmel/studio/7.0/toolchain/arm/arm-gnu-toolchain/bin/../lib/gcc/arm-none-eabi/6.3.1/thumb/v6-m/crti.o
 .ARM.attributes
                0x0000001e       0x2c c:/program files (x86)/atmel/studio/7.0/toolchain/arm/arm-gnu-toolchain/bin/../lib/gcc/arm-none-eabi/6.3.1/thumb/v6-m/crtbegin.o
 .ARM.attributes
                0x0000004a       0x32 atmel_start.o
 .ARM.attributes
                0x0000007c       0x32 Device_Startup/startup_samd21.o
 .ARM.attributes
                0x000000ae       0x32 driver_init.o
 .ARM.attributes
                0x000000e0       0x32 hal/src/hal_atomic.o
 .ARM.attributes
                0x00000112       0x32 hal/src/hal_spi_m_sync.o
 .ARM.attributes
                0x00000144       0x32 hal/src/hal_timer.o
 .ARM.attributes
                0x00000176       0x32 hal/src/hal_usb_device.o
 .ARM.attributes
                0x000001a8       0x32 hal/utils/src/utils_assert.o
 .ARM.attributes
                0x000001da       0x32 hal/utils/src/utils_list.o
 .ARM.attributes
                0x0000020c       0x32 hpl/core/hpl_init.o
 .ARM.attributes
                0x0000023e       0x32 hpl/gclk/hpl_gclk.o
 .ARM.attributes
                0x00000270       0x32 hpl/pm/hpl_pm.o
 .ARM.attributes
                0x000002a2       0x32 hpl/rtc/hpl_rtc.o
 .ARM.attributes
                0x000002d4       0x32 hpl/sercom/hpl_sercom.o
 .ARM.attributes
                0x00000306       0x32 hpl/sysctrl/hpl_sysctrl.o
 .ARM.attributes
                0x00000338       0x32 hpl/usb/hpl_usb.o
 .ARM.attributes
                0x0000036a       0x32 main.o
 .ARM.attributes
                0x0000039c       0x2c c:/program files (x86)/atmel/studio/7.0/toolchain/arm/arm-gnu-toolchain/bin/../lib/gcc/arm-none-eabi/6.3.1/../../../../arm-none-eabi/lib/thumb/v6-m\libc_nano.a(lib_a-init.o)
 .ARM.attributes
                0x000003c8       0x2c c:/program files (x86)/atmel/studio/7.0/toolchain/arm/arm-gnu-toolchain/bin/../lib/gcc/arm-none-eabi/6.3.1/../../../../arm-none-eabi/lib/thumb/v6-m\libc_nano.a(lib_a-memcpy-stub.o)
 .ARM.attributes
                0x000003f4       0x2c c:/program files (x86)/atmel/studio/7.0/toolchain/arm/arm-gnu-toolchain/bin/../lib/gcc/arm-none-eabi/6.3.1/../../../../arm-none-eabi/lib/thumb/v6-m\libc_nano.a(lib_a-memset.o)
 .ARM.attributes
                0x00000420       0x1e c:/program files (x86)/atmel/studio/7.0/toolchain/arm/arm-gnu-toolchain/bin/../lib/gcc/arm-none-eabi/6.3.1/thumb/v6-m/crtn.o

.comment        0x00000000       0x59
 .comment       0x00000000       0x59 atmel_start.o
                                 0x5a (size before relaxing)
 .comment       0x00000059       0x5a Device_Startup/startup_samd21.o
 .comment       0x00000059       0x5a driver_init.o
 .comment       0x00000059       0x5a hal/src/hal_atomic.o
 .comment       0x00000059       0x5a hal/src/hal_spi_m_sync.o
 .comment       0x00000059       0x5a hal/src/hal_timer.o
 .comment       0x00000059       0x5a hal/src/hal_usb_device.o
 .comment       0x00000059       0x5a hal/utils/src/utils_assert.o
 .comment       0x00000059       0x5a hal/utils/src/utils_list.o
 .comment       0x00000059       0x5a hpl/core/hpl_init.o
 .comment       0x00000059       0x5a hpl/gclk/hpl_gclk.o
 .comment       0x00000059       0x5a hpl/pm/hpl_pm.o
 .comment       0x00000059       0x5a hpl/rtc/hpl_rtc.o
 .comment       0x00000059       0x5a hpl/sercom/hpl_sercom.o
 .comment       0x00000059       0x5a hpl/sysctrl/hpl_sysctrl.o
 .comment       0x00000059       0x5a hpl/usb/hpl_usb.o
 .comment       0x00000059       0x5a main.o

.debug_info     0x00000000    0x2c21c
 .debug_info    0x00000000      0x38f atmel_start.o
 .debug_info    0x0000038f     0x3a43 Device_Startup/startup_samd21.o
 .debug_info    0x00003dd2     0xb24a driver_init.o
 .debug_info    0x0000f01c      0x1d1 hal/src/hal_atomic.o
 .debug_info    0x0000f1ed      0x9c9 hal/src/hal_spi_m_sync.o
 .debug_info    0x0000fbb6      0xb91 hal/src/hal_timer.o
 .debug_info    0x00010747     0x1e1a hal/src/hal_usb_device.o
 .debug_info    0x00012561      0x107 hal/utils/src/utils_assert.o
 .debug_info    0x00012668      0x314 hal/utils/src/utils_list.o
 .debug_info    0x0001297c      0x6a0 hpl/core/hpl_init.o
 .debug_info    0x0001301c      0x679 hpl/gclk/hpl_gclk.o
 .debug_info    0x00013695      0xcd7 hpl/pm/hpl_pm.o
 .debug_info    0x0001436c     0x2058 hpl/rtc/hpl_rtc.o
 .debug_info    0x000163c4     0xb266 hpl/sercom/hpl_sercom.o
 .debug_info    0x0002162a     0x1a33 hpl/sysctrl/hpl_sysctrl.o
 .debug_info    0x0002305d     0x85b4 hpl/usb/hpl_usb.o
 .debug_info    0x0002b611      0xc0b main.o

.debug_abbrev   0x00000000     0x2c3b
 .debug_abbrev  0x00000000       0xf3 atmel_start.o
 .debug_abbrev  0x000000f3      0x227 Device_Startup/startup_samd21.o
 .debug_abbrev  0x0000031a      0x3b6 driver_init.o
 .debug_abbrev  0x000006d0      0x144 hal/src/hal_atomic.o
 .debug_abbrev  0x00000814      0x1b1 hal/src/hal_spi_m_sync.o
 .debug_abbrev  0x000009c5      0x221 hal/src/hal_timer.o
 .debug_abbrev  0x00000be6      0x486 hal/src/hal_usb_device.o
 .debug_abbrev  0x0000106c       0x86 hal/utils/src/utils_assert.o
 .debug_abbrev  0x000010f2      0x152 hal/utils/src/utils_list.o
 .debug_abbrev  0x00001244      0x1d9 hpl/core/hpl_init.o
 .debug_abbrev  0x0000141d      0x1c3 hpl/gclk/hpl_gclk.o
 .debug_abbrev  0x000015e0      0x211 hpl/pm/hpl_pm.o
 .debug_abbrev  0x000017f1      0x3ed hpl/rtc/hpl_rtc.o
 .debug_abbrev  0x00001bde      0x593 hpl/sercom/hpl_sercom.o
 .debug_abbrev  0x00002171      0x25c hpl/sysctrl/hpl_sysctrl.o
 .debug_abbrev  0x000023cd      0x5ea hpl/usb/hpl_usb.o
 .debug_abbrev  0x000029b7      0x284 main.o

.debug_loc      0x00000000    0x115e7
 .debug_loc     0x00000000       0x20 atmel_start.o
 .debug_loc     0x00000020       0x78 Device_Startup/startup_samd21.o
 .debug_loc     0x00000098     0x1c98 driver_init.o
 .debug_loc     0x00001d30       0x13 hal/src/hal_atomic.o
 .debug_loc     0x00001d43      0x728 hal/src/hal_spi_m_sync.o
 .debug_loc     0x0000246b      0x767 hal/src/hal_timer.o
 .debug_loc     0x00002bd2     0x11a4 hal/src/hal_usb_device.o
 .debug_loc     0x00003d76      0x213 hal/utils/src/utils_list.o
 .debug_loc     0x00003f89       0x4c hpl/core/hpl_init.o
 .debug_loc     0x00003fd5      0x27c hpl/gclk/hpl_gclk.o
 .debug_loc     0x00004251      0x11b hpl/pm/hpl_pm.o
 .debug_loc     0x0000436c      0x561 hpl/rtc/hpl_rtc.o
 .debug_loc     0x000048cd     0x7d95 hpl/sercom/hpl_sercom.o
 .debug_loc     0x0000c662      0x2d6 hpl/sysctrl/hpl_sysctrl.o
 .debug_loc     0x0000c938     0x4b71 hpl/usb/hpl_usb.o
 .debug_loc     0x000114a9      0x13e main.o

.debug_aranges  0x00000000      0xaa0
 .debug_aranges
                0x00000000       0x20 atmel_start.o
 .debug_aranges
                0x00000020       0x28 Device_Startup/startup_samd21.o
 .debug_aranges
                0x00000048       0x58 driver_init.o
 .debug_aranges
                0x000000a0       0x30 hal/src/hal_atomic.o
 .debug_aranges
                0x000000d0       0x88 hal/src/hal_spi_m_sync.o
 .debug_aranges
                0x00000158       0x70 hal/src/hal_timer.o
 .debug_aranges
                0x000001c8      0x100 hal/src/hal_usb_device.o
 .debug_aranges
                0x000002c8       0x20 hal/utils/src/utils_assert.o
 .debug_aranges
                0x000002e8       0x48 hal/utils/src/utils_list.o
 .debug_aranges
                0x00000330       0x20 hpl/core/hpl_init.o
 .debug_aranges
                0x00000350       0x28 hpl/gclk/hpl_gclk.o
 .debug_aranges
                0x00000378       0x30 hpl/pm/hpl_pm.o
 .debug_aranges
                0x000003a8       0x70 hpl/rtc/hpl_rtc.o
 .debug_aranges
                0x00000418      0x508 hpl/sercom/hpl_sercom.o
 .debug_aranges
                0x00000920       0x28 hpl/sysctrl/hpl_sysctrl.o
 .debug_aranges
                0x00000948      0x138 hpl/usb/hpl_usb.o
 .debug_aranges
                0x00000a80       0x20 main.o

.debug_ranges   0x00000000      0xcf0
 .debug_ranges  0x00000000       0x10 atmel_start.o
 .debug_ranges  0x00000010       0x18 Device_Startup/startup_samd21.o
 .debug_ranges  0x00000028       0x48 driver_init.o
 .debug_ranges  0x00000070       0x20 hal/src/hal_atomic.o
 .debug_ranges  0x00000090       0x78 hal/src/hal_spi_m_sync.o
 .debug_ranges  0x00000108       0x90 hal/src/hal_timer.o
 .debug_ranges  0x00000198      0x108 hal/src/hal_usb_device.o
 .debug_ranges  0x000002a0       0x10 hal/utils/src/utils_assert.o
 .debug_ranges  0x000002b0       0x38 hal/utils/src/utils_list.o
 .debug_ranges  0x000002e8       0x10 hpl/core/hpl_init.o
 .debug_ranges  0x000002f8       0x18 hpl/gclk/hpl_gclk.o
 .debug_ranges  0x00000310       0x20 hpl/pm/hpl_pm.o
 .debug_ranges  0x00000330       0x60 hpl/rtc/hpl_rtc.o
 .debug_ranges  0x00000390      0x6c8 hpl/sercom/hpl_sercom.o
 .debug_ranges  0x00000a58       0x18 hpl/sysctrl/hpl_sysctrl.o
 .debug_ranges  0x00000a70      0x270 hpl/usb/hpl_usb.o
 .debug_ranges  0x00000ce0       0x10 main.o

.debug_macro    0x00000000    0x177e2
 .debug_macro   0x00000000      0x532 atmel_start.o
 .debug_macro   0x00000532      0x89e atmel_start.o
 .debug_macro   0x00000dd0      0x16d atmel_start.o
 .debug_macro   0x00000f3d       0x22 atmel_start.o
 .debug_macro   0x00000f5f       0x87 atmel_start.o
 .debug_macro   0x00000fe6       0x51 atmel_start.o
 .debug_macro   0x00001037       0xef atmel_start.o
 .debug_macro   0x00001126       0x6a atmel_start.o
 .debug_macro   0x00001190      0x1df atmel_start.o
 .debug_macro   0x0000136f       0x22 atmel_start.o
 .debug_macro   0x00001391       0x3f atmel_start.o
 .debug_macro   0x000013d0       0x1c atmel_start.o
 .debug_macro   0x000013ec       0x22 atmel_start.o
 .debug_macro   0x0000140e       0xb5 atmel_start.o
 .debug_macro   0x000014c3      0x3ad atmel_start.o
 .debug_macro   0x00001870      0x67e atmel_start.o
 .debug_macro   0x00001eee      0x8b1 atmel_start.o
 .debug_macro   0x0000279f      0x22e atmel_start.o
 .debug_macro   0x000029cd      0xd5c atmel_start.o
 .debug_macro   0x00003729      0x4dc atmel_start.o
 .debug_macro   0x00003c05      0x9f6 atmel_start.o
 .debug_macro   0x000045fb      0x82b atmel_start.o
 .debug_macro   0x00004e26      0x45f atmel_start.o
 .debug_macro   0x00005285       0x5e atmel_start.o
 .debug_macro   0x000052e3      0x8f9 atmel_start.o
 .debug_macro   0x00005bdc      0x21c atmel_start.o
 .debug_macro   0x00005df8      0x7eb atmel_start.o
 .debug_macro   0x000065e3       0x5e atmel_start.o
 .debug_macro   0x00006641      0x663 atmel_start.o
 .debug_macro   0x00006ca4      0x3ac atmel_start.o
 .debug_macro   0x00007050      0xc76 atmel_start.o
 .debug_macro   0x00007cc6     0x1092 atmel_start.o
 .debug_macro   0x00008d58      0xc4a atmel_start.o
 .debug_macro   0x000099a2      0x6ba atmel_start.o
 .debug_macro   0x0000a05c     0x1b3d atmel_start.o
 .debug_macro   0x0000bb99     0x143c atmel_start.o
 .debug_macro   0x0000cfd5      0x340 atmel_start.o
 .debug_macro   0x0000d315       0x7c atmel_start.o
 .debug_macro   0x0000d391       0xa0 atmel_start.o
 .debug_macro   0x0000d431       0x4c atmel_start.o
 .debug_macro   0x0000d47d       0xca atmel_start.o
 .debug_macro   0x0000d547       0x94 atmel_start.o
 .debug_macro   0x0000d5db       0x58 atmel_start.o
 .debug_macro   0x0000d633      0x364 atmel_start.o
 .debug_macro   0x0000d997       0x82 atmel_start.o
 .debug_macro   0x0000da19      0x189 atmel_start.o
 .debug_macro   0x0000dba2       0xb8 atmel_start.o
 .debug_macro   0x0000dc5a       0xa0 atmel_start.o
 .debug_macro   0x0000dcfa       0xb8 atmel_start.o
 .debug_macro   0x0000ddb2       0x1c atmel_start.o
 .debug_macro   0x0000ddce       0x1c atmel_start.o
 .debug_macro   0x0000ddea       0x1c atmel_start.o
 .debug_macro   0x0000de06       0x82 atmel_start.o
 .debug_macro   0x0000de88      0x15a atmel_start.o
 .debug_macro   0x0000dfe2       0x10 atmel_start.o
 .debug_macro   0x0000dff2       0xdc atmel_start.o
 .debug_macro   0x0000e0ce      0x124 atmel_start.o
 .debug_macro   0x0000e1f2      0x124 atmel_start.o
 .debug_macro   0x0000e316      0x124 atmel_start.o
 .debug_macro   0x0000e43a      0x124 atmel_start.o
 .debug_macro   0x0000e55e      0x124 atmel_start.o
 .debug_macro   0x0000e682       0xe2 atmel_start.o
 .debug_macro   0x0000e764       0xe2 atmel_start.o
 .debug_macro   0x0000e846       0xe2 atmel_start.o
 .debug_macro   0x0000e928      0x130 atmel_start.o
 .debug_macro   0x0000ea58      0x106 atmel_start.o
 .debug_macro   0x0000eb5e       0xfa atmel_start.o
 .debug_macro   0x0000ec58      0x40f atmel_start.o
 .debug_macro   0x0000f067       0x40 atmel_start.o
 .debug_macro   0x0000f0a7      0x361 atmel_start.o
 .debug_macro   0x0000f408     0x101b atmel_start.o
 .debug_macro   0x00010423       0x7b atmel_start.o
 .debug_macro   0x0001049e       0x10 atmel_start.o
 .debug_macro   0x000104ae       0x10 atmel_start.o
 .debug_macro   0x000104be       0x16 atmel_start.o
 .debug_macro   0x000104d4       0x16 atmel_start.o
 .debug_macro   0x000104ea       0x16 atmel_start.o
 .debug_macro   0x00010500       0x16 atmel_start.o
 .debug_macro   0x00010516       0x16 atmel_start.o
 .debug_macro   0x0001052c       0x16 atmel_start.o
 .debug_macro   0x00010542       0x16 atmel_start.o
 .debug_macro   0x00010558       0x16 atmel_start.o
 .debug_macro   0x0001056e       0x16 atmel_start.o
 .debug_macro   0x00010584       0x16 atmel_start.o
 .debug_macro   0x0001059a       0x16 atmel_start.o
 .debug_macro   0x000105b0       0x16 atmel_start.o
 .debug_macro   0x000105c6       0x16 atmel_start.o
 .debug_macro   0x000105dc       0x16 atmel_start.o
 .debug_macro   0x000105f2      0x4c3 atmel_start.o
 .debug_macro   0x00010ab5       0x94 atmel_start.o
 .debug_macro   0x00010b49       0x16 atmel_start.o
 .debug_macro   0x00010b5f       0x6a atmel_start.o
 .debug_macro   0x00010bc9      0x28c atmel_start.o
 .debug_macro   0x00010e55      0x4d8 atmel_start.o
 .debug_macro   0x0001132d       0x16 atmel_start.o
 .debug_macro   0x00011343       0xca atmel_start.o
 .debug_macro   0x0001140d       0x1c atmel_start.o
 .debug_macro   0x00011429       0x16 atmel_start.o
 .debug_macro   0x0001143f       0xb2 atmel_start.o
 .debug_macro   0x000114f1       0xc9 atmel_start.o
 .debug_macro   0x000115ba       0xd1 atmel_start.o
 .debug_macro   0x0001168b       0xee atmel_start.o
 .debug_macro   0x00011779      0x2e8 Device_Startup/startup_samd21.o
 .debug_macro   0x00011a61       0x39 Device_Startup/startup_samd21.o
 .debug_macro   0x00011a9a      0x552 driver_init.o
 .debug_macro   0x00011fec       0x42 driver_init.o
 .debug_macro   0x0001202e      0x416 hal/src/hal_atomic.o
 .debug_macro   0x00012444      0x46c hal/src/hal_spi_m_sync.o
 .debug_macro   0x000128b0      0x45c hal/src/hal_timer.o
 .debug_macro   0x00012d0c      0x4fe hal/src/hal_usb_device.o
 .debug_macro   0x0001320a       0xcb hal/src/hal_usb_device.o
 .debug_macro   0x000132d5       0x58 hal/src/hal_usb_device.o
 .debug_macro   0x0001332d       0x35 hal/src/hal_usb_device.o
 .debug_macro   0x00013362       0x9c hal/src/hal_usb_device.o
 .debug_macro   0x000133fe       0x58 hal/src/hal_usb_device.o
 .debug_macro   0x00013456       0x1f hal/src/hal_usb_device.o
 .debug_macro   0x00013475       0x43 hal/src/hal_usb_device.o
 .debug_macro   0x000134b8       0x20 hal/src/hal_usb_device.o
 .debug_macro   0x000134d8      0x187 hal/src/hal_usb_device.o
 .debug_macro   0x0001365f      0x34d hal/src/hal_usb_device.o
 .debug_macro   0x000139ac       0x10 hal/src/hal_usb_device.o
 .debug_macro   0x000139bc       0x35 hal/src/hal_usb_device.o
 .debug_macro   0x000139f1      0x41f hal/utils/src/utils_assert.o
 .debug_macro   0x00013e10       0x10 hal/utils/src/utils_assert.o
 .debug_macro   0x00013e20      0x423 hal/utils/src/utils_list.o
 .debug_macro   0x00014243      0x490 hpl/core/hpl_init.o
 .debug_macro   0x000146d3       0x2e hpl/core/hpl_init.o
 .debug_macro   0x00014701      0x6ec hpl/core/hpl_init.o
 .debug_macro   0x00014ded      0x432 hpl/gclk/hpl_gclk.o
 .debug_macro   0x0001521f      0x1f3 hpl/gclk/hpl_gclk.o
 .debug_macro   0x00015412      0x455 hpl/pm/hpl_pm.o
 .debug_macro   0x00015867      0x45a hpl/rtc/hpl_rtc.o
 .debug_macro   0x00015cc1       0x64 hpl/rtc/hpl_rtc.o
 .debug_macro   0x00015d25      0x65d hpl/sercom/hpl_sercom.o
 .debug_macro   0x00016382       0x70 hpl/sercom/hpl_sercom.o
 .debug_macro   0x000163f2       0x94 hpl/sercom/hpl_sercom.o
 .debug_macro   0x00016486       0x10 hpl/sercom/hpl_sercom.o
 .debug_macro   0x00016496       0x1c hpl/sercom/hpl_sercom.o
 .debug_macro   0x000164b2       0x22 hpl/sercom/hpl_sercom.o
 .debug_macro   0x000164d4       0x10 hpl/sercom/hpl_sercom.o
 .debug_macro   0x000164e4      0x42c hpl/sysctrl/hpl_sysctrl.o
 .debug_macro   0x00016910      0x2da hpl/sysctrl/hpl_sysctrl.o
 .debug_macro   0x00016bea      0x6c6 hpl/usb/hpl_usb.o
 .debug_macro   0x000172b0      0x532 main.o

.debug_line     0x00000000     0xdb94
 .debug_line    0x00000000      0xaee atmel_start.o
 .debug_line    0x00000aee      0x6e0 Device_Startup/startup_samd21.o
 .debug_line    0x000011ce      0xd87 driver_init.o
 .debug_line    0x00001f55      0x974 hal/src/hal_atomic.o
 .debug_line    0x000028c9      0xaf2 hal/src/hal_spi_m_sync.o
 .debug_line    0x000033bb      0xb12 hal/src/hal_timer.o
 .debug_line    0x00003ecd      0xd30 hal/src/hal_usb_device.o
 .debug_line    0x00004bfd      0x93e hal/utils/src/utils_assert.o
 .debug_line    0x0000553b      0x9d7 hal/utils/src/utils_list.o
 .debug_line    0x00005f12      0xa1f hpl/core/hpl_init.o
 .debug_line    0x00006931      0x9d8 hpl/gclk/hpl_gclk.o
 .debug_line    0x00007309      0x9e4 hpl/pm/hpl_pm.o
 .debug_line    0x00007ced      0xb7c hpl/rtc/hpl_rtc.o
 .debug_line    0x00008869     0x28c5 hpl/sercom/hpl_sercom.o
 .debug_line    0x0000b12e      0xa70 hpl/sysctrl/hpl_sysctrl.o
 .debug_line    0x0000bb9e     0x14e6 hpl/usb/hpl_usb.o
 .debug_line    0x0000d084      0xb10 main.o

.debug_str      0x00000000    0x82fba
 .debug_str     0x00000000    0x7339c atmel_start.o
                              0x7384c (size before relaxing)
 .debug_str     0x0007339c     0x1091 Device_Startup/startup_samd21.o
                              0x6a9d0 (size before relaxing)
 .debug_str     0x0007442d     0x1657 driver_init.o
                              0x75cf1 (size before relaxing)
 .debug_str     0x00075a84       0x9c hal/src/hal_atomic.o
                              0x724ac (size before relaxing)
 .debug_str     0x00075b20      0x2f6 hal/src/hal_spi_m_sync.o
                              0x72e46 (size before relaxing)
 .debug_str     0x00075e16      0x2d2 hal/src/hal_timer.o
                              0x72deb (size before relaxing)
 .debug_str     0x000760e8     0x3462 hal/src/hal_usb_device.o
                              0x766ad (size before relaxing)
 .debug_str     0x0007954a       0x2a hal/utils/src/utils_assert.o
                              0x724bc (size before relaxing)
 .debug_str     0x00079574       0x31 hal/utils/src/utils_list.o
                              0x72566 (size before relaxing)
 .debug_str     0x000795a5     0x17d7 hpl/core/hpl_init.o
                              0x7409b (size before relaxing)
 .debug_str     0x0007ad7c      0x855 hpl/gclk/hpl_gclk.o
                              0x72ddf (size before relaxing)
 .debug_str     0x0007b5d1      0x194 hpl/pm/hpl_pm.o
                              0x72c17 (size before relaxing)
 .debug_str     0x0007b765      0x50a hpl/rtc/hpl_rtc.o
                              0x72fc2 (size before relaxing)
 .debug_str     0x0007bc6f     0x481d hpl/sercom/hpl_sercom.o
                              0x78008 (size before relaxing)
 .debug_str     0x0008048c     0x1372 hpl/sysctrl/hpl_sysctrl.o
                              0x73a19 (size before relaxing)
 .debug_str     0x000817fe     0x1799 hpl/usb/hpl_usb.o
                              0x78795 (size before relaxing)
 .debug_str     0x00082f97       0x23 main.o
                              0x73af6 (size before relaxing)

.debug_frame    0x00000000     0x1c84
 .debug_frame   0x00000000       0x28 atmel_start.o
 .debug_frame   0x00000028       0x40 Device_Startup/startup_samd21.o
 .debug_frame   0x00000068       0xdc driver_init.o
 .debug_frame   0x00000144       0x40 hal/src/hal_atomic.o
 .debug_frame   0x00000184      0x188 hal/src/hal_spi_m_sync.o
 .debug_frame   0x0000030c      0x13c hal/src/hal_timer.o
 .debug_frame   0x00000448      0x30c hal/src/hal_usb_device.o
 .debug_frame   0x00000754       0x20 hal/utils/src/utils_assert.o
 .debug_frame   0x00000774       0x88 hal/utils/src/utils_list.o
 .debug_frame   0x000007fc       0x28 hpl/core/hpl_init.o
 .debug_frame   0x00000824       0x30 hpl/gclk/hpl_gclk.o
 .debug_frame   0x00000854       0x40 hpl/pm/hpl_pm.o
 .debug_frame   0x00000894       0xf4 hpl/rtc/hpl_rtc.o
 .debug_frame   0x00000988      0xe9c hpl/sercom/hpl_sercom.o
 .debug_frame   0x00001824       0x30 hpl/sysctrl/hpl_sysctrl.o
 .debug_frame   0x00001854      0x394 hpl/usb/hpl_usb.o
 .debug_frame   0x00001be8       0x28 main.o
 .debug_frame   0x00001c10       0x2c c:/program files (x86)/atmel/studio/7.0/toolchain/arm/arm-gnu-toolchain/bin/../lib/gcc/arm-none-eabi/6.3.1/../../../../arm-none-eabi/lib/thumb/v6-m\libc_nano.a(lib_a-init.o)
 .debug_frame   0x00001c3c       0x28 c:/program files (x86)/atmel/studio/7.0/toolchain/arm/arm-gnu-toolchain/bin/../lib/gcc/arm-none-eabi/6.3.1/../../../../arm-none-eabi/lib/thumb/v6-m\libc_nano.a(lib_a-memcpy-stub.o)
 .debug_frame   0x00001c64       0x20 c:/program files (x86)/atmel/studio/7.0/toolchain/arm/arm-gnu-toolchain/bin/../lib/gcc/arm-none-eabi/6.3.1/../../../../arm-none-eabi/lib/thumb/v6-m\libc_nano.a(lib_a-memset.o)
